:1000000000000120750300005D0300005F03000095
:1000100061030000630300006503000000000000AE
:100020000000000000000000000000006703000066
:1000300069030000000000006B0300006D03000076
:100040006F0300006F0300006F0300006F030000E8
:100050006F0300006F0300006F0300006F030000D8
:100060006F0300006F0300006F0300006F030000C8
:100070006F0300006F0300006F0300006F030000B8
:100080006F0300006F0300006F0300006F030000A8
:100090006F0300006F0300006F0300006F03000098
:1000A0006F0300006F0300006F0300006F03000088
:1000B0006F0300006F03000000000000000000005C
:1000C0006F0300006F0300006F0300006F03000068
:1000D0006F0300006F0300006F03000000000000CA
:1000E0000000000000000000000000000000000010
:1000F0000000000000000000000000000000000000
:1001000000000000000000000000000000000000EF
:1001100000000000000000000000000000000000DF
:1001200000000000000000000000000000000000CF
:1001300000000000000000000000000000000000BF
:1001400000000000000000000000000000000000AF
:10015000000000000000000000000000000000009F
:10016000000000000000000000000000000000008F
:10017000000000000000000000000000000000007F
:10018000000000000000000000000000000000006F
:10019000000000000000000000000000000000005F
:1001A000000000000000000000000000000000004F
:1001B000000000000000000000000000000000003F
:1001C000000000000000000000000000000000002F
:1001D000000000000000000000000000000000001F
:1001E000000000000000000000000000000000000F
:1001F00000000000000000000000000000000000FF
:10020000354936480A1A02D0072291438D463449AF
:1002100034480A1A06D00722914381F30988022242
:1002200082F3148830483149314A00F044F83148AB
:100230003149324A00F03FF831483249324A00F041
:100240003AF832483249334A00F035F832483349F7
:10025000334A00F030F833483349344A00F02BF881
:1002600033483449344A00F026F8344834490022EF
:1002700000F02CF833483449002200F027F83348C6
:100280003349091A082902DB002202604160314A21
:1002900090471F481F49884205D00268043003B4C4
:1002A000904703BCF7E700208646EC46002000217B
:1002B000294A9047FEE7884207D0521A05D00378B2
:1002C00001300B700131013AF9D17047884202D0F8
:1002D00002700130FAE770470000012000E00020C2
:1002E00000000120000001205C0700000000002049
:1002F00004000020D0030000D003000040070000ED
:100300005C07000000000020000000204007000003
:1003100040070000400700004007000040070000C1
:100320004007000040070000400700005C07000095
:1003300060070000040000200400002004000020EA
:10034000040000200400002004000020040000201D
:10035000042000209D0300002D040000FEE7FEE7BE
:10036000FEE7FEE7FEE7FEE7FEE7FEE7FEE7FEE765
:1003700000F002B8FFF7FCBF0F484FF007018843B9
:1003800085460E4880470E48016841F470010160BF
:10039000BFF34F8FBFF36F8FFFF732BF09480A4992
:1003A0000A4A884207D0521A05D0037801300B70F0
:1003B0000131013AF9D1704700000120A904000081
:1003C00088ED00E040070000000000200000002051
:1003D0004FF0A0434FF40042C3F8082570474FF098
:1003E000A042D2F80435D94301F4004103F400439C
:1003F000C2F80815C2F80C357047C20708B506D513
:100400004FF0A0430322C3F83C27FFF7E1FF830727
:100410000AD54FF0A0430C22C3F83427C3F838277D
:10042000C3F83C27C3F8402708BD000008B50120E9
:10043000074CFFF7E2FF44F001040020FFF7CFFF75
:100440004FF4FA754FF47A40A047013DFAD1F4E732
:10045000400700004FF08053D3F83001421C04BF26
:100460004FF0704393F8E00F831F58425841704794
:100470004FF0704393F8E02F062A09D1D3F8E83FF4
:10048000C3F30313033B042B02D8024AD05C70472A
:100490000020704755070000024AD2F80034002BB4
:1004A000FBD0704700E0014010B5FFF7D3FF40B12B
:1004B0004FF08053944AD3F82433C3F30423C2F893
:1004C0004035FFF7D5FF10B1904B914A5A67FFF7BF
:1004D000C1FF48B14FF080534FF08042D3F844320F
:1004E000C3F34233C2F83C35FFF7C2FF30B1894A4B
:1004F000D2F8FC3023F08073C2F8FC30FFF7AAFF7B
:1005000040B14FF080430022C3F80C21C3F8102102
:10051000C3F83825FFF7ACFF20B14FF0804303222A
:10052000C3F8A025FFF7A4FF60B17B4B0522C3F8F9
:1005300010260122C3F888260022C3F818263F227D
:10054000C3F814264FF08053D3F83021511C09BF53
:100550004FF07043D3F8343193F8E02FD3F8E83FED
:1005600008BFC3F30313062A4DD1033B042B03D862
:100570006A4AD35C002B46D04FF08052684BD2F8C9
:100580000414C3F82015D2F80814C3F82415D2F8BF
:100590000C14C3F82815D2F81014C3F82C15D2F88F
:1005A0001414C3F83015D2F81814C3F83415D2F85F
:1005B0001C14C3F84015D2F82014C3F84415D2F81F
:1005C0002414C3F84815D2F82814C3F84C15D2F8EF
:1005D0002C14C3F85015D2F83014C3F85415D2F8BF
:1005E0003414C3F86015D2F83814C3F86415D2F87F
:1005F0003C14C3F86815D2F84014C3F86C15D2F84F
:100600004424C3F87025FFF725FF48B14FF080530D
:100610004FF08042D3F8583203F04F03C2F8E43E63
:10062000FFF718FF48B14FF08043D3F80024D207FA
:1006300044BF6FF00102C3F800244FF08053D3F899
:100640003021062A0ED1D3F83431033B042B02D8D3
:10065000344AD35C33B1344AD2F83C3743F4806334
:10066000C2F83C372B4AD2F8883043F47003C2F802
:100670008830BFF34F8FBFF36F8F4FF08053D3F8A5
:100680003021062A0FD1D3F83431033B042B02D892
:10069000264AD35C3BB14FF01023D3F808224FF029
:1006A0008043C3F858254FF01023D3F80022002AC6
:1006B00003DBD3F80432002B22DA1D4901234FF06B
:1006C0001020C1F804351524FFF7E6FEC0F80042FB
:1006D000FFF7E2FEC0F80442FFF7DEFE0023C1F898
:1006E0000435FFF7D9FEBFF34F8F0A49114BCA6893
:1006F00002F4E0621343CB60BFF34F8F00BFFDE70E
:100700000D4B0E4A1A6010BD0030014000C007407A
:100710000DF0ADBA00ED00E00050004046070000CB
:1007200000C000404B0700000010004050070000D0
:1007300000E001400400FA05000000200090D00312
:100740000338FDD8704700000101010000000101DD
:0C0750000000000001010000000000009B
:04075C000090D00336
:040000030000037581
:00000001FF
